:0800000000008A110A12052814
:06000A000430FE0001308D
:10001000FF0080308A110A12E3208A110A1283122B
:100020000313A1007F08A0000630A2000130A30046
:10003000831203132008A4002108A500FF30A007A5
:10004000031CA10324082504031995280430220762
:10005000A400A501A50D2308A5072408FE00250876
:10006000FF0080308A110A12E3208A110A128312DB
:100070000313A7007F08A6002208FE002308FF0044
:1000800080308A110A12E3208A110A1283120313A4
:10009000A900A5007F08A800A40002302207A40040
:1000A000A501A50D2308A5072408FE002508FF00CB
:1000B00080308A110A12E3208A110A128312031374
:1000C000A500AB007F08A400AA0083120313260832
:1000D000AA002708AB00FF30A607031CA7032A08C5
:1000E0002B0403198E282808FE002908FF00803001
:1000F0008A110A12D0208A110A1283120313AA004D
:10010000240884008313251883172A088000A80A6E
:100110000319A90AA40A0319A50A6528063083123F
:100120000313A2070318A30A18288A110A12992890
:100130000800831603138610C220831203138C1E3B
:100140009D281A0883120313AE0083120313AC0117
:1001500083120313861CAF2883120313AC0A0130E9
:1001600083120313AC062C08AD002D0C0318BB281A
:10017000831203138610031CC028831203138614F2
:100180009D28080083160313181581309900181252
:100190008312031398171816831603139816080072
:1001A000003A0319D728803A0319DE2800347E0864
:1001B000840083137F188317000808007F088A00D3
:1001C0007E0882000800003A0319EB28803A0319E0
:1001D000F528FF0100347E08840083137F188317FD
:1001E0000008FF00840A000808008A110A12DE20B5
:1001F000FD00FE0FFF03FF0A8A110A12DE20FC0039
:100200007D08FF007C080800013400340C34013400
:0A0210002F340034013400340034B0
:00000001FF
